:020000040000fa
:080000000002040000000000f2
:020000040000fa
:100400000f80200000ff2000000188000000000095
:100410000c000700e0e721000100200011000700a8
:10042000000020000000e000020032000000020096
:1004300000000000b40b0200000000000040da00e1
:100440000000fe004440a900409220000000e000af
:100450000300320000002000a00188004440a800f2
:100460000000060091018800800078000000eb0089
:1004700015003700e280400032a0b4009101ba00bc
:10048000e280400032a0b4009102ba00e280400055
:1004900032a0b4000002eb00472bde00f507b200eb
:1004a000602ce10004003a000059eb008301e900f0
:1004b000fdff3e00040037006128e100010032002a
:1004c0000082eb00040007001101ba000200e00006
:1004d000e8ff3a00000006003159ba008301e90044
:1004e0000c0032002159ba008301e90008003200f3
:1004f0000400e00003003a00e280400032a0b400b3
:10050000f5ff370011d9ba008301e900faff3a007c
:100510008100e800e180400032a0b4000000060045
:020000040000fa
:0200000401f009
:040010007eff00006f
:020000040000fa
:0200000401f009
:040014007fff00006a
:020000040000fa
:0200000401f009
:04001800ffff0000e6
:020000040000fa
:0200000401f009
:04001c00dfff000002
:020000040000fa
:10000800801e0000801e0000801e0000801e000070
:10001800801e0000801e0000801e0000801e000060
:10002800801e0000801e0000801e0000801e000050
:10003800801e0000801e0000801e0000801e000040
:020000040000fa
:020000040000fa
:1005200000000000ffff0000ffff0000ffff0000d1
:10053000ffff0000ffff000001000000ffff0000c0
:10054000ffff0000ffff00000100000001000000ad
:10055000ffff0000ffff0000ffff0000ffff0000a3
:1005600001000000ffff0000ffff0000010000008d
:100570000100000001000000ffff0000ffff00007d
:1005800001000000ffff000001000000ffff00006d
:1005900001000000ffff000001000000010000005a
:1005a000ffff0000ffff0000ffff0000ffff000053
:1005b0000100000001000000ffff0000010000003a
:1005c000010000000100000001000000ffff00002a
:1005d00001000000ffff0000ffff0000010000001d
:1005e00001000000ffff000001000000010000000a
:1005f00001000000ffff0000ffff000001000000fd
:10060000ffff0000ffff0000ffff000001000000ef
:10061000ffff000001000000ffff0000ffff0000df
:10062000ffff0000ffff000001000000ffff0000cf
:1006300001000000ffff00000100000001000000b9
:10064000ffff000001000000ffff0000ffff0000af
:100650000100000001000000010000000100000096
:100660000100000001000000ffff00000100000089
:1006700001000000ffff0000ffff0000010000007c
:10068000ffff0000ffff000001000000ffff00006f
:10069000ffff000001000000ffff0000010000005c
:1006a00001000000ffff0000010000000100000049
:1006b0000100000001000000010000000100000036
:1006c000ffff0000ffff000001000000ffff00002f
:1006d000ffff00000100000001000000ffff00001c
:1006e00001000000ffff000001000000ffff00000c
:1006f000ffff00000100000001000000ffff0000fc
:10070000ffff00000100000001000000ffff0000eb
:10071000ffff0000ffff0000ffff0000ffff0000e1
:10072000ffff0000ffff00000100000001000000cb
:10073000ffff0000ffff0000ffff000001000000be
:1007400001000000ffff0000ffff000001000000ab
:10075000ffff000001000000ffff0000ffff00009e
:10076000ffff00000100000001000000ffff00008b
:1007700001000000ffff0000ffff0000010000007b
:10078000ffff000001000000010000000100000068
:100790000100000001000000010000000100000055
:1007a000ffff000001000000ffff0000ffff00004e
:1007b000ffff000001000000ffff0000010000003b
:1007c00001000000ffff0000ffff0000ffff00002e
:1007d000010000000100000001000000ffff000018
:1007e00001000000ffff0000010000000100000008
:1007f000ffff0000ffff000001000000ffff0000fe
:100800000100000001000000ffff0000ffff0000ea
:1008100001000000010000000100000001000000d4
:10082000ffff0000ffff0000ffff000001000000cd
:1008300001000000010000000100000001000000b4
:10084000ffff0000010000000100000001000000a7
:10085000ffff000001000000ffff0000ffff00009d
:10086000ffff0000ffff0000ffff0000010000008d
:1008700001000000ffff000001000000ffff00007a
:100880000100000001000000ffff00000100000067
:1008900001000000ffff0000010000000100000057
:1008a00001000000ffff0000010000000100000047
:1008b000ffff0000ffff0000ffff0000ffff000040
:1008c000ffff000001000000ffff0000010000002a
:1008d00001000000ffff000001000000ffff00001a
:1008e0000100000001000000010000000100000004
:1008f00001000000ffff000001000000ffff0000fa
:1009000001000000ffff000001000000ffff0000e9
:1009100001000000ffff0000ffff0000ffff0000dc
:10092000ffff0000ffff0000ffff000001000000cc
:10093000ffff000001000000ffff0000ffff0000bc
:1009400001000000ffff000001000000ffff0000a9
:100950000100000001000000010000000100000093
:10096000ffff0000ffff000001000000ffff00008c
:10097000010000000100000001000000ffff000076
:10098000010000000100000001000000ffff000066
:10099000ffff0000ffff0000ffff0000ffff00005f
:1009a000ffff000001000000010000000100000046
:1009b000ffff0000ffff0000010000000100000039
:1009c00001000000ffff000001000000ffff000029
:1009d000ffff000001000000ffff0000ffff00001c
:1009e0000100000001000000010000000100000003
:1009f000ffff000001000000ffff000001000000f9
:100a00000100000001000000ffff000001000000e5
:100a1000ffff000001000000ffff0000ffff0000db
:100a2000ffff000001000000ffff0000ffff0000cb
:100a300001000000ffff0000ffff0000ffff0000bb
:100a4000ffff00000100000001000000ffff0000a8
:100a5000ffff000001000000010000000100000095
:100a6000ffff0000ffff0000ffff0000ffff00008e
:100a700001000000ffff0000010000000100000075
:100a80000100000001000000ffff00000100000065
:100a900001000000ffff0000010000000100000055
:100aa000ffff0000ffff0000010000000100000048
:100ab000ffff000001000000ffff0000ffff00003b
:100ac000ffff0000ffff0000010000000100000028
:100ad00001000000ffff0000010000000100000015
:100ae0000100000001000000ffff0000ffff000008
:100af000ffff0000ffff00000100000001000000f8
:100b000001000000010000000100000001000000e1
:100b1000010000000100000001000000ffff0000d4
:100b2000ffff0000ffff0000ffff0000ffff0000cd
:100b300001000000010000000100000001000000b1
:100b4000ffff0000010000000100000001000000a4
:100b50000100000001000000ffff0000ffff000097
:100b6000ffff000001000000ffff00000100000087
:100b70000100000001000000ffff0000ffff000077
:100b80000100000001000000ffff0000ffff000067
:100b900001000000ffff0000ffff0000ffff00005a
:100ba000ffff0000ffff000001000000ffff00004a
:100bb000ffff000001000000ffff00000100000037
:100bc000ffff0000ffff0000010000000100000027
:100bd00001000000ffff0000010000000100000014
:100be000ffff000001000000ffff0000ffff00000a
:100bf000ffff0000010000000100000001000000f4
:100c000001000000ffff0000ffff000001000000e6
:100c100001000000010000000100000001000000d0
:100c2000ffff0000ffff00000100000001000000c6
:100c3000ffff00000100000001000000ffff0000b6
:100c4000ffff0000ffff000001000000ffff0000a9
:100c500001000000ffff000001000000ffff000096
:100c6000ffff000001000000ffff0000ffff000089
:100c7000ffff000001000000010000000100000073
:100c8000ffff0000ffff0000ffff00000100000069
:100c900001000000ffff0000010000000100000053
:100ca000ffff000001000000ffff00000100000046
:100cb000ffff000001000000010000000100000033
:100cc000ffff0000ffff0000ffff00000100000029
:100cd000ffff0000ffff0000010000000100000016
:100ce000ffff0000ffff0000ffff00000100000009
:100cf000ffff0000ffff0000ffff000001000000f9
:100d0000ffff0000ffff0000ffff0000ffff0000eb
:100d1000ffff0000ffff0000ffff0000ffff0000db
:100d200001000000000000000000000000000000c2
:100d3000000000000000000000000000ffff0000b5
:100d4000010000000000000000000000ffff0000a4
:100d50000000000001000000000000000000000092
:100d600000000000ffff0000010000000000000084
:100d7000ffff000000000000000000000100000074
:100d800000000000ffff000001000000ffff000066
:100d900001000000ffff000001000000ffff000055
:100da0000000000001000000000000000000000042
:100db00000000000ffff0000000000000100000034
:100dc000ffff000000000000000000000000000025
:100dd00001000000ffff0000010000000000000013
:100de000ffff00000000000001000000ffff000006
:100df00000000000000000000100000000000000f2
:100e0000ffff0000010000000000000000000000e3
:100e1000ffff000001000000ffff000001000000d4
:100e2000000000000000000000000000ffff0000c4
:100e300001000000ffff000001000000ffff0000b4
:100e40000000000001000000ffff000001000000a2
:100e500000000000ffff0000000000000000000094
:100e60000000000000000000000000000100000081
:100e7000ffff000000000000010000000000000073
:100e8000ffff00000100000000000000ffff000065
:100e90000100000000000000ffff00000100000052
:100ea000ffff00000000000001000000ffff000045
:100eb0000000000000000000000000000000000032
:100ec000000000000100000000000000ffff000023
:100ed0000100000000000000ffff00000000000013
:100ee00001000000ffff000001000000ffff000004
:100ef0000100000000000000ffff000000000000f3
:100f00000100000000000000ffff000000000000e2
:100f100001000000000000000000000000000000d0
:100f2000000000000000000000000000ffff0000c3
:100f300000000000010000000000000000000000b0
:100f4000ffff0000000000000100000000000000a2
:100f5000ffff000001000000ffff00000100000093
:100f60000000000000000000ffff00000000000083
:100f700001000000ffff0000010000000000000071
:100f8000ffff000001000000ffff00000000000064
:100f90000000000000000000000000000000000051
:100fa0000000000001000000ffff00000100000041
:100fb0000000000000000000ffff00000100000032
:100fc000ffff000000000000010000000000000022
:100fd00000000000ffff0000000000000000000013
:100fe00001000000ffff000001000000ffff000003
:100ff000000000000100000000000000ffff0000f2
:1010000001000000ffff00000000000001000000e0
:1010100000000000ffff00000000000000000000d2
:1010200000000000010000000000000000000000bf
:10103000ffff0000000000000000000000000000b2
:101040000000000001000000ffff000000000000a1
:101050000000000001000000ffff00000100000090
:101060000000000000000000000000000000000080
:10107000ffff00000000000001000000ffff000073
:1010800001000000ffff0000000000000100000060
:10109000ffff00000000000001000000ffff000053
:1010a000000000000000000001000000ffff000041
:1010b000000000000100000000000000000000002f
:1010c0000000000000000000ffff00000100000021
:1010d000ffff00000000000001000000ffff000013
:1010e00001000000ffff0000000000000000000001
:1010f000000000000000000001000000ffff0000f1
:1011000001000000ffff000001000000ffff0000e1
:1011100001000000ffff00000100000000000000cf
:1011200000000000000000000000000000000000bf
:10113000ffff000001000000ffff000001000000b1
:1011400000000000ffff000001000000ffff0000a2
:1011500001000000ffff0000000000000000000090
:10116000000000000100000000000000ffff000080
:1011700001000000ffff0000000000000000000070
:1011800001000000ffff0000000000000000000060
:10119000010000000000000000000000000000004e
:1011a0000000000000000000ffff00000000000041
:1011b000000000000100000000000000ffff000030
:1011c000000000000000000001000000ffff000020
:1011d0000100000000000000ffff0000010000000f
:1011e00000000000ffff0000000000000000000001
:1011f0000000000001000000ffff000001000000ef
:10120000ffff0000000000000000000001000000df
:10121000ffff000001000000ffff000001000000d0
:101220000000000000000000ffff000001000000bf
:1012300000000000ffff00000100000000000000af
:101240000000000000000000ffff000000000000a0
:101250000100000000000000ffff0000000000008f
:10126000000000000100000000000000000000007d
:1012700000000000ffff000001000000ffff000071
:10128000000000000000000000000000010000005d
:10129000ffff00000000000001000000ffff000051
:1012a000000000000100000000000000ffff00003f
:1012b0000000000001000000ffff0000010000002e
:1012c000000000000000000000000000ffff000020
:1012d000000000000000000001000000ffff00000f
:1012e00000000000000000000000000001000000fd
:1012f000000000000000000000000000ffff0000f0
:1013000000000000000000000000000000000000dd
:1013100000000000000000000000000000000000cd
:1013200001000000000000000000000000000000bc
:1013300000000000ffff00000000000000000000af
:101340000000000001000000ffff0000000000009e
:10135000000000000000000000000000010000008c
:101360000000000000000000ffff0000010000007e
:10137000ffff00000000000000000000010000006e
:1013800000000000ffff000000000000010000005e
:1013900000000000ffff000001000000000000004e
:1013a000000000000000000000000000ffff00003f
:1013b0000100000000000000ffff0000010000002d
:1013c000ffff00000100000000000000ffff000020
:1013d000000000000000000001000000ffff00000e
:1013e0000000000001000000ffff000001000000fd
:1013f0000000000000000000ffff000000000000ef
:1014000000000000000000000100000000000000db
:10141000ffff0000000000000000000000000000ce
:10142000000000000100000000000000ffff0000bd
:101430000000000001000000ffff000000000000ad
:10144000010000000000000000000000ffff00009d
:1014500001000000ffff000001000000ffff00008e
:101460000100000000000000ffff0000010000007c
:101470000000000000000000ffff0000000000006e
:10148000000000000100000000000000000000005b
:10149000ffff00000000000001000000ffff00004f
:1014a0000000000001000000ffff0000010000003c
:1014b000ffff000001000000ffff0000000000002f
:1014c000000000000100000000000000000000001b
:1014d000ffff00000100000000000000ffff00000f
:1014e00000000000010000000000000000000000fb
:1014f000ffff0000010000000000000000000000ed
:10150000ffff0000010000000000000000000000dc
:1015100000000000000000000000000000000000cb
:1015200000000000000000000001000002020000b6
:10153000030300000303000004040000040400008f
:101540000404000004040000050500000505000077
:101550000505000005050000050500000505000063
:10156000050500000505000006060000060600004f
:10157000060600000606000006060000060600003b
:10158000060600000606000006060000060600002b
:10159000060600000606000006060000060600001b
:1015a0000606000006060000070700000707000007
:1015b00007070000070700000707000007070000f3
:1015c00007070000070700000707000007070000e3
:1015d00007070000070700000707000007070000d3
:1015e00007070000070700000707000007070000c3
:1015f00007070000070700000707000007070000b3
:1016000007070000070700000707000007070000a2
:101610000707000007070000070700000707000092
:10162000070700000707000008080000080800007e
:10163000080800000808000008080000080800006a
:10164000080800000808000008080000080800005a
:10165000080800000808000008080000080800004a
:10166000080800000808000008080000080800003a
:10167000080800000808000008080000080800002a
:10168000080800000808000008080000080800001a
:10169000080800000808000008080000080800000a
:1016a00008080000080800000808000008080000fa
:1016b00008080000080800000808000008080000ea
:1016c00008080000080800000808000008080000da
:1016d00008080000080800000808000008080000ca
:1016e00008080000080800000808000008080000ba
:1016f00008080000080800000808000008080000aa
:101700000808000008080000080800000808000099
:101710000808000008080000080800000808000089
:1017200008080000080800003031000032330000d3
:1017300034350000363700003839000041420000df
:10174000434400004546000000ff00000100000087
:101750000100000000ff0000ff0000000001000089
:0817600000010000ff00000081
:020000040000fa
:101768001e04fa00b0052000303a880044c7bf00c4
:10177800f043b20044e7b70041742000914078007c
:1017880000ceb30000c060006040b30044e7b7007b
:10179800103a80004800de00405f98004e589000e4
:1017a8008080fb00800f2000008060006300400004
:1017b8000001780081072000a00920003374200070
:1017c800814978008049780082497800103a800081
:1017d800405f98004e5890000004a0000081fb0074
:1017e80061042000700520002374200081497800de
:1017f800804978008249780042c7bf000042b200a1
:101808000004e000fcff320042c7bf0061406000f6
:101818000004e000fcff3a00a016200040118800f8
:101828000080280000118800004024001011880062
:10183800e0ff2f0060198800c05e200000198800b2
:10184800e0002000101988005132200091407800f3
:1018580000ceb30000c060006040b30025e3b700cd
:1018680080c0b30024e3b70025e3a9000000eb0023
:101878004019880021e3a800103a8000405f9800d2
:101888004e5890008080fb00f00b20000081600023
:10189800610420007005200023742000814978002d
:1018a8008049780082497800f16c200091407800e6
:1018b80000ceb30000c060002041b300cfe6b700ff
:1018c800716c20009140780000ceb30000c0600029
:1018d8003041b300c7e6b700616c20009140780042
:1018e80000ceb30000c060003040b300c6e6b700c9
:1018f800ce58900000c4b30000c070000081fb0007
:1019080061042000700520002374200081497800bc
:10191800804978008249780060002000200c880007
:1019280000042000000c8800e0002000500c880013
:1019380000202000300c8800000028008008880063
:101948000000eb0030088800f03f200060088800a5
:1019580000002800900888000000eb00500888006c
:10196800f03f200070088800c422a900cc42a900da
:10197800cc62a800cca2a900cd02a900cd22a90062
:10198800cd42a900cd62a900cd82a900cda2a800b0
:10199800cdc2a900c022a900c082a900c842a900de
:1019a800c862a900c882a900c8a2a900c902a900e2
:1019b800c922a900c942a900c962a900c982a9000f
:1019c800c9a2a900c9c2a9006880a80068a0a80087
:1019d8000040eb00405f9800140037004e5890001c
:1019e8000082fb004e5890008080fb00a316200068
:1019f8008e814100018140000000eb0000b17900b8
:101a0800a21620000e01410001804000600179000b
:101a1800a10720008e8040000400420002b0780038
:101a28004e5890000040e800405f9800ce58900063
:101a380070c7b30080cf5000e8ff36000040eb00cd
:101a4800405f9800260037004e5890008082fb00c7
:101a58004e5890000082fb004e5890008080fb009a
:101a6800a02d20000e004000808040000040eb00c8
:101a7800804878004e5890008080fb00a3312000f9
:101a88008e814100018140000000eb0000b1790027
:101a9800a23120000e014100018040006001790060
:101aa800a13920008e8040000400420002b0780076
:101ab800a13920008e804000040042006080780038
:101ac80000017800a12520008e804000058042009a
:101ad80002b078004e5890000040e800405f98003f
:101ae800ce589000f0c3b30080cf5000d6ff360028
:101af8006000b80070379800013f98007e30900071
:101b08008e389000103f9800213f98000040eb006d
:101b180000ef98000000eb0050379800de3090008e
:101b280061379800f00f2000602f98000040eb000c
:101b380000df98000000eb00502f98000040eb00f9
:101b4800306f98000040eb0070d798000040eb0021
:101b580060d7980022c3bf000080fb004700de006a
:101b68000080fb0060179800f00f2000102f9800ed
:101b78001e299000022f98000000eb00202f9800eb
:101b8800ae299000732798000000eb0040279800ca
:101b9800000420003027980030f2200070179800c9
:101ba8000040eb00307798000000eb00001f980021
:101bb80010c0b300507798000040eb0040779800c1
:101bc8006000b80040079800510798004e00900048
:101bd800de0090006007980071079800d0ff2f0082
:101be800000f780030f220001007980000c0eb00ca
:101bf800005798000040eb00207f98000040eb0061
:101c0800206f9800700880004600dd000100200069
:101c1800301f9800411f98006000b8001017980006
:101c2800211798001e119000ae11900032179800ed
:101c3800431798000040eb00705f9800fe59900031
:101c4800036798000040eb00605f98000080eb009d
:101c58008080eb0000279800112798000080eb0097
:101c68008080eb00601f9800711f980020052000fd
:101c78002011880030052000201188004005200030
:101c8800201188000000370022c3bf000080fb003d
:101c98004700de008080fb006e109000808f5000af
:101ca800f9ff320022c3bf000080fb004700de00be
:101cb8000080fb00601798006e1090000000e000a4
:101cc80036003a008018800080007800a018800054
:101cd80000805000403f98009018800080007800f5
:101ce800b018800000805000303f980080188000b5
:101cf80080007800806b2000808f500023003c001b
:101d0800801880008000780080942f00808f500019
:101d18001e0035009018800080007800806b20003d
:101d2800808f500019003c009018800080007800d7
:101d380080942f00808f500014003500a018800078
:101d480080007800806b2000808f50000f003c00de
:101d5800a01880008000780080942f00808f5000a9
:101d68000a003500b018800080007800806b2000e1
:101d7800808f500005003c00b0188000800078007b
:101d880080942f00808f500039003d004e20900035
:101d98000000e80040279800350037000018800050
:101da800800078002018800000805000403f980094
:101db80010188000800078003018800000805000e3
:101dc800303f98000018800080007800806b200069
:101dd800808f500023003c000018800080007800ad
:101de80080942f00808f50001e003500101880004e
:101df80080007800806b2000808f500019003c0024
:101e0800101880008000780080942f00808f500088
:101e1800140035002018800080007800806b2000b6
:101e2800808f50000f003c00201880008000780050
:101e380080942f00808f50000a00350030188000f1
:101e480080007800806b2000808f500005003c00e7
:101e5800301880008000780080942f00808f500018
:101e680003003d004e2090000000e8004027980045
:101e78000ee890000080fb00a11620008e80400034
:101e880000004000e08078003e38900001005000db
:101e98006101b9007e3090008e389000000041004a
:101ea8008180490070379800013f98000ee8900043
:101eb8000080fb00a11620008e804000000040003a
:101ec8003e39900002b078000ee890000080fb00d8
:101ed800a10720008e80400000004000e0807800cc
:101ee8004e389000010050006101b9001e38900082
:101ef800ae3890000000410081804900103f9800f2
:101f0800213f98000ee890000080fb00a107200008
:101f18008e80400000004000ce39900003b0780069
:101f28000ee890000040e80000ef98008ee890006e
:101f380080c7b30080cf500002003a000040eb0099
:101f480000ef98007e3090008e3890004c09dd003c
:101f58004400de0000007100c488de00503798009d
:101f68001e389000ae389000cc09dd004400de0039
:101f780000807100c488de00603798000e20900051
:101f88009e209000e00f5000e08f580006003500ba
:101f98000e2090009e20900061004000e0804800e4
:101fa80000279800112798000e2190009e2190008c
:101fb800c0eb220011002000800f5100818f5900d2
:101fc80003003a006000b800002798001127980025
:101fd800cac2bf00614060000004e0000b0032008c
:101fe8006e199000fe1990000080eb008080eb00d5
:101ff800800f5100818f590004003a000e20900094
:102008009e209000601f9800711f9800cac2bf00f0
:10201800614060000004e00004003a000080eb002a
:102028008080eb00601f9800711f98007e10900060
:102038000000e900701798007e1090000000e00092
:1020480032003a0030f22000701798000041eb008f
:10205800b14120008e804000824878002e709000a8
:102068000004e00004003a0010c0b300b3412000af
:102078008e81410080497800b14120008e80400067
:1020880091407800217798008e189000700c2000fd
:10209800808f5000080034003e7090000004e0007b
:1020a80002003a000040eb00605f980010c0b300e7
:1020b80030779800060037005e5890000004e00072
:1020c800030032000e1890000000e800001f98007e
:1020d8003e7090000004e0000b0032002e7090006b
:1020e80061406000614060004401dd00412c200037
:1020f80091407800f0ceb30000c06000024070004c
:10210800c4e2b70001003700c482a9003e6890000d
:102118000040e800306f9800be689000d0c4b3005b
:1021280080cf500002003a000040eb00306f98006a
:102138006e3090000000e000030035006e31900022
:102148002237980004003700ee3090000080eb0042
:102158000088b900203798005e3090000000e00049
:1021680003003500de319000333798000400370053
:10217800de3090000080eb000088b900303798000e
:10218800be3090002e30900000804000c800de0075
:1021980040a928000080400090407800415f9800e6
:1021a8004e5890008080fb002e3090000100de0029
:1021b800203798004e5890008080fb003e309000f9
:1021c8000100de0030379800ae3090002e309000cd
:1021d8000088b90000017800be3090003e309000c1
:1021e8000088b90000004100103798000000eb009b
:1021f8000037980000002400702f9800fe289000f7
:102208001e309000808f50002d0036007e289000f0
:102218004200de00702f9800fe2890001e309000cb
:10222800808f5000260036007e2890004200de0095
:10223800702f9800fe2890001e309000808f50006c
:102248001f0036007e2890004200de00702f9800a4
:10225800fe2890001e309000808f50001800360035
:102268007e2890004200de00702f9800fe28900023
:102278001e309000808f5000110036007e2890009c
:102288004200de00702f9800fe2890001e3090005b
:10229800808f50000a0036007e2890004200de0041
:1022a800702f9800fe2890001e309000808f5000fc
:1022b800030036007e2890004200de00702f980050
:1022c8007e2890000000e000da0032008e30900096
:1022d8007e289000808040001e309000808f500043
:1022e8000c003e008e3090007e28900080804000d8
:1022f8001e30900001005000103798000e309000fa
:102308008000d1007e2890000080400000379800af
:10231800030037000e3090000000d100003798000d
:102328007e2890004200de00702f98007e289000e2
:102338000000e000bf0032008e3090007e28900040
:10234800808040001e309000808f50000c003e00be
:102358008e3090007e289000808040001e309000d3
:1023680001005000103798000e3090008000d10016
:102378007e28900000804000003798000300370056
:102388000e3090000000d100003798007e289000a1
:102398004200de00702f98007e2890000000e000c8
:1023a800a40032008e3090007e289000808040008b
:1023b8001e309000808f50000c003e008e30900040
:1023c8007e289000808040001e3090000100500060
:1023d800103798000e3090008000d1007e289000c1
:1023e8000080400000379800030037000e3090004e
:1023f8000000d100003798007e2890004200de00df
:10240800702f98007e2890000000e00089003200bc
:102418008e3090007e289000808040001e30900012
:10242800808f50000c003e008e3090007e28900077
:10243800808040001e309000010050001037980046
:102448000e3090008000d1007e289000008040006f
:1024580000379800030037000e3090000000d100cc
:10246800003798007e2890004200de00702f980008
:102478007e2890000000e0006e0032008e30900050
:102488007e289000808040001e309000808f500091
:102498000c003e008e3090007e2890008080400026
:1024a8001e30900001005000103798000e30900048
:1024b8008000d1007e2890000080400000379800fe
:1024c800030037000e3090000000d100003798005c
:1024d8007e2890004200de00702f98007e28900031
:1024e8000000e000530032008e3090007e289000fb
:1024f800808040001e309000808f50000c003e000d
:102508008e3090007e289000808040001e30900021
:1025180001005000103798000e3090008000d10064
:102528007e289000008040000037980003003700a4
:102538000e3090000000d100003798007e289000ef
:102548004200de00702f98007e2890000000e00016
:10255800380032008e3090007e2890008080400045
:102568001e309000808f50000c003e008e3090008e
:102578007e289000808040001e30900001005000ae
:10258800103798000e3090008000d1007e2890000f
:102598000080400000379800030037000e3090009c
:1025a8000000d100003798007e2890004200de002d
:1025b800702f98007e2890000000e0001d00320077
:1025c8008e3090007e289000808040001e30900061
:1025d800808f50000c003e008e3090007e289000c6
:1025e800808040001e309000010050001037980095
:1025f8000e3090008000d1007e28900000804000be
:1026080000379800030037000e3090000000d1001a
:10261800003798007e2890004200de00702f980056
:102628007e2890000000e000020032000000eb006d
:10263800702f98004e589000e74f500003003a0062
:102648000e319000622f9800100037004e5890000d
:10265800e74f5000070036004e5890000080fb00fe
:10266800e70050000e3090000100dd00602f980058
:10267800060037004e5890000080fb00e70010006d
:102688000e3090000100de00602f9800ee289000c8
:102698000e289000808f500002003600cc82a800df
:1026a80005003700ee2890007e209000808f5000b3
:1026b80001003100cc82a900ee28900070022000b1
:1026c800808f500002003c0010c0b3005077980083
:1026d8001e0090000000e900100798001e00780016
:1026e800c34120008e81410080097800c14120004b
:1026f8008e80400091007800e18f40004900320050
:10270800c24120000e01410012017800e10f410092
:1027180010003c00c34120008e81410093017800e5
:10272800e38f410021003200c04120000e0040002c
:1027380010007800e30f40002e003c00c14120004b
:102748008e80400091007800ea8f4000130032002c
:102758005703370010202000c24120000e0141001d
:1027680012017800800f51006a00320020202000fa
:10277800c34120008e81410093017800808f510071
:102788008e023200c04120000e0040001000780088
:102798000000e00036003200450337001e009000bc
:1027a8000000e800100798008703370000c0eb001e
:1027b80000579800ccc2bf00704060000004e000e1
:1027c800030032003e7090000004e00002003a006e
:1027d80030f22000100798001e0090000000e00072
:1027e80079033a0010002000100798001e0fe80037
:1027f80075033700ccc2bf00704060000004e000e1
:1028080004003a0030f22000100798001e0fe8007c
:102818006d0337001e0090000000e80010079800c4
:10282800690337001e0090000000e00004003a0031
:1028380030d22200100798001e0fe800620337000c
:10284800ccc2bf00704060000004e00003003a0002
:102858003e7090000004e0005b033a0030f2200074
:1028680010079800d0ff2f00000f7800560337009c
:102878001e0090000000e00010003a00cd02a90000
:102888006000b80020079800310798002e019000da
:10289800be01900062079800730798006e009000d0
:1028a800fe0090004007980051079800800720001c
:1028b800100798001e0fe800430337009e009000a1
:1028c80080d62200808f50003f033e000e509000bb
:1028d8000004e0003c033400ccc2bf000080fb00d1
:1028e8004400de000004a200614060006140600016
:1028f8006140600061416000d12c20009140780067
:10290800e0cfb30000c0600002407000cde2b70025
:102918002d0337009e009000a0052000808f5000f6
:1029280014003a006e009000fe009000e00f500086
:10293800e08f58000f003d00ce0090000080eb00b3
:10294800000ab800ce0090000080eb000088b900b3
:102958000501780000014100de0090000080eb00d6
:102968000088b900000141008202780044079800fd
:10297800550798009e00900000052000808f5000a9
:102988001a003a003e7090000080fb00e1006000f1
:1029980040b928000080400090407800a02d200019
:1029a8000e004000014878006e009000fe00900084
:1029b8004109dd004f00de0000007100cf88de0015
:1029c800610160006000b800030020000200700090
:1029d8008380700042b928000200400090407800cf
:1029e800a02d20000e004000114098009e0090008d
:1029f80060042000808f500019003a00ee219000fa
:102a0800430f9800ce089000f00f2000808f5000f0
:102a180002003600f00f2000400f98004e0890008a
:102a28004400de00ef00600040b92800008040004c
:102a380090407800a02d20000e0040002140980012
:102a48004e089000ef00600040b928000080400068
:102a580090407800a02d20000e00400031409800e2
:102a68009e009000c0032000808f50005a003a005a
:102a78006e009000fe009000100f9800210f980043
:102a88001e099000ae099000f0ff27000100200009
:102a9800800f5100818f590004003400f0ff270097
:102aa80001002000100f9800210f98001e099000c7
:102ab800ae09900000002800f1ff2f00800f5100a0
:102ac800818f590004003d0000002800f1ff2f000d
:102ad800100f9800210f98001e089000ae08900073
:102ae8004409dd004c00de0000007100cc88de00e7
:102af8006f0160006000b800030020000200700051
:102b08008380700042b9280002004000904078009d
:102b1800a02d20000e004000414098001e089000a3
:102b2800ae089000c809dd004800de000080710092
:102b3800c888de006f0160006000b8000300200054
:102b4800020070008380700042b928000200400033
:102b580090407800a02d20000e00400051409800c1
:102b68001e089000ae0890004c09dd004400de000d
:102b780000007100c488de006f0160006000b800ca
:102b880003002000020070008380700042b9280012
:102b98000200400090407800a02d20000e00400068
:102ba800614098001e089000ae0890006f01600018
:102bb8006000b800030020000200700083807000ed
:102bc80042b928000200400090407800a02d200063
:102bd8000e004000714098009e00900020032000e5
:102be800808f50005a003a004e009000de0090009e
:102bf800100f9800210f98001e099000ae09900050
:102c0800f0ff270001002000800f5100818f59003c
:102c180004003400f0ff270001002000100f980086
:102c2800210f98001e099000ae09900000002800ae
:102c3800f1ff2f00800f5100818f590004003d00e3
:102c480000002800f1ff2f00100f9800210f9800b6
:102c58001e089000ae0890004409dd004c00de001c
:102c680000007100cc88de006f0160006000b800d1
:102c780003002000020070008380700042b9280021
:102c88000200400090407800a02d20000e00400077
:102c9800014898001e089000ae089000c809dd00a1
:102ca8004800de0000807100c888de006f01600007
:102cb8006000b800030020000200700083807000ec
:102cc80042b928000200400090407800a02d200062
:102cd8000e004000114898001e089000ae089000b1
:102ce8004c09dd004400de0000007100c488de00ed
:102cf8006f0160006000b80003002000020070004f
:102d08008380700042b9280002004000904078009b
:102d1800a02d20000e004000214898001e089000b9
:102d2800ae0890006f0160006000b800030020004a
:102d3800020070008380700042b928000200400041
:102d480090407800a02d20000e00400031489800e7
:102d58009e00900080022000808f500021003a00e1
:102d68003e189000ce189000c909dd004700de002b
:102d780000807100c788de00400f98004e08900060
:102d88004800de00ef00600040b9280000804000e5
:102d980090407800a02d20000e0040004148980087
:102da8004e0890004400de00ef00600040b92800a3
:102db8000080400090407800a02d20000e004000c8
:102dc800514898004e089000ef00600040b9280074
:102dd8000080400090407800a02d20000e004000a8
:102de800614898001e009000fe0f50001c003a0039
:102df8003e209000400f98004e0890004800de00ea
:102e0800ef00600040b92800008040009040780042
:102e1800a02d20000e004000714898004e08900038
:102e28004400de00ef00600040b928000080400048
:102e380090407800a02d20000e004000015098001e
:102e48004e089000ef00600040b928000080400064
:102e580090407800a02d20000e00400011509800ee
:102e68001e009000f40f500018003a002e00900049
:102e7800be0090004709dd004900de000000710037
:102e8800c988de00400f98004e0890004400de001c
:102e9800ef00600040b928000080400090407800b2
:102ea800a02d20000e004000215098004e089000f0
:102eb800ef00600040b92800008040009040780092
:102ec800a02d20000e004000315098001e009000f8
:102ed800ea0f500053003a004e019000de019000c6
:102ee800007d200001002000800f5100818f5900d3
:102ef80015003c004e019000de01900000832f0079
:102f0800f1ff2f00800f5100818f59000e0035000e
:102f18006e019000fe019000f07c2000010020006e
:102f2800800f5100818f59001b003c006e019000fa
:102f3800fe01900000832f00f1ff2f00800f510049
:102f4800818f5900140034000e5090000004e000f6
:102f5800040034000e5090000040e900005798002b
:102f68003000370010002000001f9800a12d20001d
:102f78008e8040000040eb00c050980010022000f6
:102f880020118800d0ff2f00000f780030f22000b9
:102f980010079800230037004e019000de019000d2
:102fa800703e200001002000800f5100818f5900e1
:102fb8001c003c004e019000de01900080c12f00f3
:102fc800f1ff2f00800f5100818f59001500340048
:102fd8006e019000fe01900080bb200001002000df
:102fe800800f5100818f590007003c006e0190004e
:102ff800fe01900080442f00f1ff2f00800f510048
:10300800818f590007003d008e509000b0c3b30077
:1030180080cf500003003c000e5090000040e800b4
:10302800005798001e009000e60f500014003a0068
:103038000e5090000000fb004480de000000fb0002
:10304800ef00600040b92800008040009040780000
:10305800a02d20000e004000415098000e50900016
:103068000000fb00ef00600040b92800008040002d
:1030780090407800a02d20000e004000515098008c
:103088001e0090000000e0004f013a000040eb00f5
:10309800605798000e5090000004e00018003d00b2
:1030a8004e009000de009000c909dd004700de00f8
:1030b80000807100c788de00500f9800de0890007d
:1030c80080072000808f50000300340080c7b300c1
:1030d800605798001f003700de08900080f82f0026
:1030e800808f500003003d0080c8b30060579800ef
:1030f800180037005e0890006057980015003700e8
:103108004e019000de019000100020000100200018
:10311800800f5100818f5900040034006e509000d8
:103128000040e800605798000a0037004e01900000
:10313800de0190000080eb008080eb00800f5100e2
:10314800818f590003003d006e5090000040e90057
:10315800605798006e5090000000fb004480de002d
:103168000000fb00ef00600040b92800008040002c
:1031780090407800a02d20000e004000615098007b
:103188006e5090000000fb00ef00600040b928007e
:103198000080400090407800a02d20000e004000e4
:1031a800715098006e5090000000fb00801bb0002a
:1031b800100798001e0fe800030137009e009000da
:1031c800d0032000808f50005f003a000e2090004e
:1031d8009e209000e00f5000e08f580004003d0052
:1031e80000002800010020000027980011279800ff
:1031f8000e2090009e2090004088de00cf80de00e8
:103208006f0160006000b800030020000200700039
:103218008380700042b92800020040009040780086
:10322800a02d20000e004000515898000e2090005c
:103238009e2090004409dd004c00de000000710073
:10324800cc88de006f0160006000b8000300200039
:10325800020070008380700042b92800020040001c
:1032680090407800a02d20000e0040006158980082
:103278000e2090009e209000c809dd004800de0066
:1032880000807100c888de006f0160006000b8002f
:1032980003002000020070008380700042b92800fb
:1032a8000200400090407800a02d20000e00400051
:1032b800715898000e2090009e2090004c09dd0067
:1032c8004400de0000007100c488de006f01600069
:1032d8006000b800030020000200700083807000c6
:1032e80042b928000200400090407800a02d20003c
:1032f8000e004000016098000e2090009e20900073
:103308006f0160006000b800030020000200700038
:103318008380700042b92800020040009040780085
:10332800a02d20000e00400011609800a12d200063
:103338008e8040000040eb00a0609800a0032000b1
:1033480020118800cd02a8001e009000ea0f50004e
:103358004f003a006e189000fe1890004088de007a
:10336800cf80de006f0160006000b800030020001d
:10337800020070008380700042b9280002004000fb
:1033880090407800a02d20000e00400001589800c1
:103398006e189000fe189000c409dd004c00de0095
:1033a80000807100cc88de006f0160006000b8000a
:1033b80003002000020070008380700042b92800da
:1033c8000200400090407800a02d20000e00400030
:1033d800115898006e189000fe1890004809dd00fa
:1033e8004800de0000007100c888de006f01600040
:1033f8006000b800030020000200700083807000a5
:1034080042b928000200400090407800a02d20001a
:103418000e004000215898006e189000fe18900089
:10342800cc09dd004400de0000807100c488de00a5
:103438006f0160006000b800030020000200700007
:103448008380700042b92800020040009040780054
:10345800a02d20000e004000315898006e189000f2
:10346800fe1890006f0160006000b80003002000a3
:10347800020070008380700042b9280002004000fa
:1034880090407800a02d20000e0040004158980080
:103498001e0090000000e0004b003a00c0c8230066
:1034a800100798000000eb00000f78004600370076
:1034b8009e009000c0032000808f500017003a0043
:1034c8006e2890000000e000140032006e3090007a
:1034d8000000e00011003d001e0078008000400060
:1034e8002069280000804000900078005e3090003d
:1034f8000088b9006e299000110009000200d80068
:103508006101b9004e009000de009000000041000b
:103518008180490040079800510798001e009000dc
:10352800fe0f50000b003a00100020009e0f100004
:10353800080034006e2890006101b9002e00900048
:10354800be009000000041008180490020079800db
:10355800310798001e0090000000e0001a003a00b1
:103568006e2890000000e000140032006e309000d9
:103578000000e00011003d001e00780080004000bf
:103588000029280000804000900078005e309000fc
:103598000088b9006e299000110009000200d800c7
:1035a8006101b9006e009000fe009000000041002b
:1035b8008180490060079800710798008007200003
:1035c800100798001e0fe8000ee890000004e000c5
:1035d8005d003a005e7090000004e0001a003a00b6
:1035e800ee28900080022000808f500016003400e2
:1035f8005e3090006e299000110009000200d8008a
:10360800500f9800de08900010f82f00808f5000af
:1036180003003d0010c8b300605798000c00370045
:10362800de089000f0072000808f5000030034006f
:10363800f0c7b30060579800050037005e08900097
:1036480060579800020037000040eb006057980070
:103658003e189000ce1890004909dd004700de00b2
:1036680000007100c788de00800078006e5090006e
:103678000000fb0000804000400f98004e089000ba
:103688006103b800be189000f00720000009b800d8
:103698003e1890006000b900030278000002420062
:1036a800ce189000f00720000088b9000002420000
:1036b800840178000200be00f003b0000180b00071
:1036c800c909dd004700de0000807100c788de0000
:1036d8000600400087804800301f9800411f98006e
:1036e8004e089000300c88000041eb00a1412000fa
:1036f8008e804000824878003e7090000004e00010
:1037080004003a0010c0b300a34120008e8141009c
:1037180080497800a14120008e80400091407800c7
:1037280061c060004301dd00c12c20009140780099
:1037380070cfb30000c0600002407000cce2b70058
:103748000040eb00507798000ee89000f04f5000d2
:1037580063003a007e5890000080fb00a1392000e9
:103768008e80400000004000e08078006e309000bd
:10377800010050006101b9003e109000ce10900089
:1037880000004100818049003017980041179800d7
:103798007e5890000080fb00a13920008e804000f8
:1037a800000040006e31900002b078007e58900012
:1037b8000080fb00a13120008e8040000000400006
:1037c800e08078005e309000010050006101b9008f
:1037d8001e109000ae10900000004100818049004a
:1037e80010179800211798007e5890000080fb0061
:1037f800a13120008e80400000004000de319000a2
:1038080003b078007e5890000040e800f043b20012
:10381800705f98000e6090000080fb004200de00a0
:10382800006798001e109000ae109000e00f500046
:10383800e08f580003003d000e6090006440400097
:10384800006798003e109000ce109000e00f5000e6
:10385800e08f580003003d000e6090006840400073
:10386800006798000e6090008080fb0040ba280036
:103878000080400090407800615798006e5090009a
:103888000004e00004003a00ee28900080022000c6
:10389800808f50000200340010c0b300505f9800c1
:1038a800ee5890006e50900000c04000605f980095
:1038b8006e589000e34f500003003c006e58900093
:1038c800e44f400006003c000040eb0030779800d1
:1038d8000000eb00001f98000040eb00605f9800bc
:1038e8003e689000e24f500011003a002e209000f0
:1038f8008000e800f03f200000806000202798004a
:103908002e2090000000e00009003a005e58900068
:103918000004e00004003a000000eb00001f9800db
:103928000040eb00307798000040eb00505f9800b3
:103938003e689000e44f50004b003a00ee2890009b
:103948005e28900001004000502f98007ed0900023
:103958000080fb00a12520008e8040000000400070
:10396800e08078002e289000808f500007003600f5
:103978007ed090000080fb00a12520008e804000b2
:103988000000400060817800222f98007ed09000cf
:103998000080fb00a12520008e8040000000400030
:1039a800e08078001e289000808f500007003100ca
:1039b8007ed090000080fb00a12520008e80400072
:1039c80000004000e0817800132f98007ed090001e
:1039d8000040e80070d798007ed090000080fb007f
:1039e800a12520008e80400000004000e080780083
:1039f8002e289000808f5000070036007ed090005f
:103a08000080fb00a12520008e80400000004000bf
:103a180060817800222f98007ed090000080fb0003
:103a2800a12520008e80400000004000e080780042
:103a38001e289000808f5000070031007ed0900033
:103a48000080fb00a12520008e804000000040007f
:103a5800e0817800132f98007ed090000040e800a5
:103a6800f043b20070d798003e689000e64f5000cf
:103a780028003a000ed89000f04f500025003a0078
:103a88004e2090000000e00006003a004e709000c2
:103a9800ef4f5000030036003e20900064004000c5
:103aa800302798004e209000e70f500003003e009a
:103ab8003e2090000000e80030279800ce209000bb
:103ac80000022000808f5000050036004e20900034
:103ad800c500de003e20900001005000302798000d
:103ae800be209000f03f2000808f5000020036007a
:103af800f03f2000302798003e209000000c8800fe
:103b08000000eb00402798000040eb004077980049
:103b18000a003700ee2890000e289000808f500091
:103b2800060036003e689000e64f500003003a0059
:103b38004e7090000040e800407798003e68900082
:103b48000004e0002f003a000ed890000040e80082
:103b580000df98000ed89000ff4f50002900360073
:103b68000040eb0000df98006ed090000081fb0061
:103b78005e289000c501de00a12520008e8040004f
:103b88000200410003b078000000eb00502f9800bd
:103b98006ed090000040e800f043b20060d7980073
:103ba800ae2890001e2890000080500060279800e2
:103bb8006e2090004200de006300b90080007800ab
:103bc8001e28900000804000002f98006e20900072
:103bd8008000d1001e2890000080400050279800e7
:103be8006e209000c200de001e2890000080400079
:103bf80070279800f00f2000102f98000000eb00ad
:103c0800202f980023c2bf00614060000004e0003c
:103c180021003a0023c2bf00624060000004e000b7
:103c28001d003a002e6890008080fb00a02d200027
:103c38000e00400000804000104078000004e000c2
:103c4800130032002e6890008080fb00a02d200019
:103c58000e00400000804000104078000080fb000b
:103c6800201188002e6890008080fb00a02d200085
:103c78000e004000808040000040eb008048780043
:103c88002e6890000040e800206f9800020037007e
:103c98000040eb00206f980022c3bf000080fb00ab
:103ca8004700de008080fb006e109000808f50007f
:103cb800f5f73200cdc2bf000080fb004500de00f2
:103cc8000004a20061406000614060006140600043
:103cd800614060004501dd00d12c20009140780052
:103ce800f0cdb30000c0600002407000cde2b70024
:043cf800e5f73700b5
:020000040000fa
:043cfc0000000000c4
:020000040000fa
:043d00000000fe00c1
:00000001FF
